:020000020000FC
:0400000004C014C064
:10000800B8C00FED0DBF00E001BB0FEB02BB0FE066
:1000180007BB02EF08BB00E40BBF789408E305BFF9
:100028008895EFCF00270BBF05BF992709E00EBDC4
:1000380003E00BBD07EE0ABD00E409BFC09AC198F2
:10004800789404E1302E15D0DCCF13D012D011D023
:1000580010D00FD00ED00DD00CD00BD00AD009D0B4
:1000680008D007D006D005D004D003D002D001D0E4
:10007800C8CFEF93FF93F0E0EAE809D0FF91EF9142
:10008800089557414B45205550200A0D0000EF9325
:10009800FF93C895002021F0002D4ED03196F9CF5E
:1000A800FF91EF9133D00895013039F08894079586
:1000B80010F01CD0F9CF1FD0F7CF0895EF93FF931E
:1000C800003211F423D00FC00B350AF00F750A3235
:1000D80052F0F1E0E8E40A52E00F0027F01FC8955B
:1000E800002DE2DF0FD0FF91EF910895926016D0B6
:1000F8009D7F14D00895926011D010D00FD09D7FAD
:100108000DD008950BD00AD009D0089507D006D095
:1001180005D004D003D002D001D008950F931F93C7
:10012800032D222414E11A95F1F72A94D9F70A9598
:10013800C1F71F910F9108950F930F91BFDF089595
:10014800682A735E7A293F3E3C3830202123272FC6
:1001580047553101014C010611150902140B100411
:100168001E0D1207050F161B0A08030C180E191D81
:1001780013010F930FB70F9391FF11C0BA9A092F6C
:1001880001700395017021F4C298C39A9E7F03C041
:10019800C29AC39891600F910FBF0F911895BA98A2
:0E01A800000000000000000000000000F4CF86
:00000001FF
